:040000000A160028B4
:10000800FF00030E8301DF000A08E4008A0170087C
:10001800A2007108A1000408A30083168C1E7A2888
:1000280083128C1E7A28981C2C281812181660081F
:10003800013EF00000300318013E6107F10070082E
:10004800E0007108E1001A080317A900A9017A283D
:100058000313181D3E286008013EF0000030031805
:10006800013E6107F1007008E0007108E100031724
:10007800A9017A2803131A080317A90029080D3AB9
:1000880003195328803003135C06F0008030700297
:10009800031D502820305B020318532862280313DD
:1000A800E5165B08C03E840080015B08DD005C0843
:1000B800DE00DB01DC010317A9017A2803135B08C2
:1000C800C03E840003172908800003135B08DD0085
:1000D8005C08DE005B08013EF00000300318013EBA
:1000E8005C07F1007008DB007108DC008B1EA0289B
:1000F8000B1DA028831203130B113C3081006208EA
:10010800013EF00000300318013E6307F10070085B
:10011800E2007108E30080306306F000803070026E
:10012800031D982864306202031CA0286515E201AB
:10013800E3018A1541268A11831203132208F0006D
:100148002108F1002308840064088A005F0E8300F8
:06015800FF0E7F0E0900FE
:10015E0083120313F201F30180307306F000803036
:10016E007002031DBC28083072020318D528031331
:10017E008711803003172805F1007108803A031D9E
:10018E00CB2803130716CD28031307128715031761
:0E019E00A80D2810F20A0319F30AB32808006E
:1001AC00831203138714071003172708A800AF2026
:0801BC0083120313071408006D
:0E01C4008312031369088A006808820008008D
:1001D200831203137008F100F0010830FC0071086B
:1001E200F40C0318F828FC0BF128F1010034031079
:1001F200FD28F40C0318F107F10CF00CFC0BFA28A3
:020202000800F2
:10020400063084000008000883120313F000701302
:06021400700880000800E4
:10021A00831203172208F2007208F000F20A70082B
:10022A008400000803191A29112922087202F00011
:0C023A000130F002F101031CF103080088
:06024600000000000800AA
:10024C00831203138710071003172208A800AF208E
:10025C00213083120313FC007630FD00FD0B342992
:0A026C00FC0B342900000714080001
:10027600063084000008000883120313F000F01310
:0602860070088000080072
:10028C007B15FB1F50290130F300F201F101F00145
:08029C00FA0DF20CFF3008001E
:0E02A400F201F101F001F801F3010030080051
:0802B200FA1FF21300300800EE
:1002BA00831603139818632900005D298312031714
:0802CA0022080313990008004B
:1002D2002030831203172202031C742922087F3C58
:1002E200031C74297529B0290530F0002208F40096
:1002F200E920A03070020317A3000030031C013E66
:100302007102A4000530A5000030A6008030F00084
:10031200803026067002031D90292508003C031830
:10032200AE292308003EF00018300318013E2407CE
:10033200F10070080313E8007108E900E2208A1155
:100342000A120317A700D6200317A30A0319A40A47
:100352000130A502031CA6038729A701D6200800A5
:100362003B218316861323212321061783126A1049
:10037200061BBF296A1CBE29BF29B92923212321B3
:10038200232123212321232123212321831686179D
:06039200232123210800D5
:100398007B14FB1FD729F201FA1FFF30F200F1008E
:0A03A800F000FA0DF20CFF3008001F
:1003B200FB14FB1FE329FF30F300F200F100F00011
:0803C200FA0DF20CFF300800F7
:1003CA00A0017208031DFA297108F2007008F100F1
:1003DA00F001A0157208031DFA297108F200F10153
:1003EA00A011201672080319082A2008F302031D17
:1003FA00031C0C2A0310F21B102AF00DF10DF20D4A
:10040A00F30B002A0C2A0130FC005221132A023075
:0E041A00FC004621132A0430FC005921080082
:10042800013083120317A0000030A10080309E0025
:100438009F011E081F0403194D2A2321232123216C
:100448002321022183160613232123218312031754
:100458001E081D05F00000301F05F100700871042A
:1004680003193A2A8316031386173D2A3B2183165C
:10047800861323212321061783126A10061B482A94
:100488006A1C472A482A422A03179F0C9E0C9F136E
:100498001D2AA001A101232123210221831606136D
:1004A80023212321861723212321232123210617F2
:1004B80083126A10061B642A6A1C632A642A5E2A4D
:1004C8000317A001A10123212321861F6C2A2014D0
:1004D80023212321232123212321232123212321F4
:1004E80023212321232123212321232123212321E4
:1004F8000221831606133B218316861383120317E2
:060508002008F0000800CD
:10050E00831203171D08A2000D2170089F009E0183
:10051E001E081D0784000008A0000313651B9C2AFB
:10052E0003172008A2005D21A02A03172008A200AD
:10053E006921831203179E0A80301E06F000803058
:0A054E001F067002031C8F2A08002C
:1005580083120313F8010830FC00700DF80D7408BD
:10056800F8020318B92AF8070310F00DFC0BB12A9A
:02057800080079
:10057A0083160313861723212321061723212321F8
:10058A003B21831686132321232102218316061376
:02059A00080057
:06059C00FB15FF30080012
:1005A200831203171E08003C0318F02A09301E02AA
:1005B2000318F02A1E03F0000730F00540307004E3
:1005C200A200262103171D08F0000630F400E920DE
:1005D2007F30F005803070040317A2002621080046
:1005E2008312031799019A0180309B0000309C000E
:1005F2001B081C0403191F2B232123218316031319
:10060200861723212321061783126A10061B0D2B3E
:100612006A1C0C2B0D2B072B861F142B03171B0890
:1006220099041C089A04232123210221831606130C
:10063200831203179C0C9B0C9C13F92A8316031339
:10064200861723212321831203171708180403197D
:100652002D2B3B218316861383160313232123217B
:10066200061783126A10061B3A2B6A1C392B3A2B87
:10067200342B232123210221831606132321232134
:100682003B2183168613831203171908F000080012
:10069200BD22D030831203179D0014227008031369
:1006A200BD0003179D01142270080313BD008030A2
:1006B20003179D00142270080313BD0024080317BA
:1006C2009D00142270080313BD003E0803179D000D
:1006D200142270080313BD00410803179D00142261
:1006E20070080313BD00400803179D001422700810
:1006F2000313BD003F0803179D0014227008031363
:10070200BD004D0803179D00142270080313BD009D
:10071200B121BD222130FC007630FD00FD0B8F2B74
:10072200FC0B8F2B0000D030831203179D00142284
:1007320070080313BD0003179D01142270080313F0
:10074200BD0003179D01142270080313BD00B121DF
:0207520008009D
:100754008312031718080313E80003171908031377
:10076400E900E2208A110A12F00070080319D02B64
:10077400031718080313E800031719080313E90003
:10078400E2208A110A12F000031717088400700887
:100794008000970A980A0319990AAA2B03171708C5
:0607A40084008001080042
:1007AA00831203136513031719089D00872200306B
:1007BA001806031DE22B01301706031DEB2B0A3026
:1007CA00A2005D210D300317A2005D2103136517F6
:0207DA00080015
:1007DC000130831203179D0001309E00D12221307D
:1007EC0083120313FC007630FD00FD0BFB2BFC0B7E
:1007FC00FB2B000003179701980180301806F000BE
:10080C008030033A7002031D0D2C003017020318C0
:10081C00202CA701D6200430FC003D30FD00FD0B40
:10082C00152CFC0B152C000000000317970A03195C
:06083C00980A032C0800DD
:100842008312031719089D0017089E00D1228312F4
:0A08520003171B08A200692108002B
:10085C00831203137008F8007108F000F101F20123
:10086C00F301FB01FC019630F300FA01F01F442C5C
:10087C00F809F009F80A0319F00AFA177008F100E0
:0C088C007808F000F801F201E5210800F6
:1008980083120313FB017308031D77080319A32CA4
:1008A80072087606FA007708F3077E30031C602C7E
:1008B800F3020318A62C632CF302031CA92C72085C
:1008C800F8007108FC007008FD00F817F61703100F
:1008D800F201F101F0011830A0007D1C7D2C740894
:1008E800F00775080318750FF10776080318760FD7
:1008F800F207F20CF10CF00CF80CFC0CFD0C0310D8
:10090800A00B712CF21B8D2CF80DF00DF10DF20DD2
:10091800F3037B1B701C9F2CF81F9F2CF00A0319F4
:10092800F10A0319F20A031D9F2CF20CF10CF00CCA
:10093800F30A0319A62CFA1FF2130030AB2C01306E
:100948005221AB2C0230D921AB2C043046210000B7
:02095800080095
:10095A0083120313FB01FA01F9018030F800F10C4C
:10096A00F00C031CC12C7408F90775080318750FDD
:10097A00FA070318FB0A0310F01FC92C7408FA07B8
:10098A0075080318750FFB07FB0CFA0CF90CF80C29
:10099A00031CB42C7B08F3007A08F2007908F100F2
:0609AA007808F0000800CF
:1009B000831203179901170884000008980018088B
:1009C000003A0319EE2C1808A2005D210317990ABA
:0E09D00019081707840000089800DF2C0800A3
:1009DE00831203137408003A031D0A2D7508003A9A
:1009EE00031D0A2D7608003A031D0A2D7708003ADA
:1009FE00031D0A2DFF30F000FF30F1007F30F200B2
:100A0E00FF30F300A52D8312031377080319992DD8
:100A1E00730803199C2D720876068039FA00F217B6
:100A2E00F617A0017208F8007108FC007008FD00AE
:100A3E007408FD027508031C750FFC027608031C72
:100A4E00760FF802F801FC01FD01031C352D031091
:100A5E00F20CF10CF00CF80C0130A0007708F30248
:100A6E00031C3F2D7E302007F30703189F2D442DC6
:100A7E007E302007F307031CA22D1830FA07FD0D58
:100A8E00FC0DF80DF00DF10DF20DA00D7408F00235
:100A9E007508031C750FF1027608031C760FF2021F
:100AAE00760DA004201C5D2D7D14682D7408F007B2
:100ABE0075080318750FF10776080318760AF20702
:100ACE007D10FA031F307A05031D462D7B1B7D1CFE
:100ADE008F2D0310F00DF10DF20DA00D7408F00224
:100AEE007508031C750FF1027608031C760FF202CF
:100AFE00760D20040139FD070318FC0A0319F80AC4
:100B0E00031D8F2DF80CFC0CFD0CF30A03199F2D01
:100B1E00FA1FF8137808F2007C08F1007D08F00047
:100B2E000030A42D0130CE22A42D02305221A42D4E
:0E0B3E000430D921A42D083046210000080003
:100B4C0083120313FB01FC01FA0173080319E52D51
:100B5C00F2178E30F302F31BB62D0319B62DE82DC8
:100B6C00F309F30A08307302031CCB2DF300F10DCB
:100B7C007208F100F20108307302031CCB2DF10D49
:100B8C00F1017308031D0310D32D73080319D32D22
:100B9C000310F20CF10CF30BCE2D7B1B711CDD2D15
:100BAC00031CDD2DF10A0319F20AF21BF42DFA1FB6
:100BBC00F72DF209F109F10A0319F20AF72DF201E6
:100BCC00F101F72D7B14FB1FFA2DF201FA1FFA2D00
:100BDC00FF30F200F100FA0DF20CFA2D0130FC009E
:100BEC00FC2D0030FC00FC2DFF30FC00FC08031930
:0E0BFC00002ECC217108F0007208F1000800F4
:100C0A00831203179901033019020318132E1908C6
:100C1A001807840020308000990A082E190818073E
:100C2A00840080019903190818079A000A30F40011
:100C3A001708F000AC227808F0003030F0070317EC
:100C4A001A088400700880000A30F4001708F000BF
:100C5A00AC227008031797007008003A031D362E5D
:080C6A00382E9903182E080032
:100C720083120313F801F9011030FC00710DF80D15
:100C8200F90D7408F8027508031C750FF9020318B0
:100C9200512E7408F80775080318750FF907031029
:0A0CA200F00DF10DFC0B3F2E0800D1
:100CAC00710DF80DF90D7408F8027508031C750F19
:100CBC00F902F00DF10D0F30FC00710DF80DF90D6E
:100CCC007408701C6F2EF8027508031C750FF9025E
:100CDC00742EF80775080318750FF907F00DF10D50
:100CEC00FC0B632E7018802E7408F8077508031817
:080CFC00750FF9070000080064
:100D0400831203136D08073C03188B2EF001F101C5
:100D1400AD2EC7309F056D08F000F00D7010F00D7A
:100D24007010F00D701070089F040A30FC00BC3085
:100D3400FD00FD0B9B2EFC0B9B2E00001F150000DD
:100D44001F1DA52EA22E1E08F100F00183161E08F9
:080D5400F0070318F10A080082
:100D5C00831203136D08E8006E08E900E2208A1183
:100D6C000A12F00070080319C92E6D08E8006E080D
:100D7C00E900E2208A110A120317A2005D21ED0A94
:080D8C000319EE0AAE2E080067
:100D9400831203171008F0001108F1002E2400300C
:100DA400F4000030F5004030F6008530F7004C24A4
:100DB4000030F4000030F5000030F6008930F70010
:100DC400EF247008C3007108C4007208C5007308DA
:100DD400C600A6257008031794007108950080309A
:100DE400F000803013067002031DFA2E1208003C36
:100DF4000318432F80301306F00080307002031D67
:100E0400052F093012020318432F1203F000073094
:100E1400F00540307004A2002621ED01EE010030FF
:100E24006E02031D172F5E306D0203183A2F8030B7
:100E34006D040317A20026216E0803171502031D73
:100E4400272F03136D0803171402031C2D2F3C30A6
:100E5400A700D620302F0317A701D6200330FD00AA
:100E6400FD0B322F00000000ED0A0319EE0A112FCA
:100E740003171203F0000730F00540307004A2009D
:040E8400262108001B
:100E880083160313EF0105306F020318542F6F0800
:100E980083126F078400203080008316EF0A472FE3
:100EA8006F0883126F07840080018316EF036F08B1
:100EB80083126F07031790000A30F400F50103133B
:100EC8006D08F0006E08F10039267808F0007908FE
:100ED800F1003030F0070317100884007008800014
:100EE8000A30F400F50103136D08F0006E08F100F4
:100EF80039267008ED007108EE0000307106031DF8
:100F0800872F00307006031D8A2F8D2F8316EF035D
:040F18005B2F080043
:100F1C00831203179D0103136D0803179E00D12242
:100F2C00213083120313FC007630FD00FD0B9C2F47
:100F3C00FC0B9C2F000001306D02F0000030031CF4
:100F4C00013E6E02F1006030F4000030F500AD247B
:100F5C00603070070317900071080318013E910070
:100F6C0070080313ED007108EE0080306E06F0007F
:100F7C008030031711067002031DC72F10080313CE
:100F8C006D020318DA2F0317A701D6200430FC00DA
:100F9C003D30FD00FD0BD02FFC0BD02F00000000CE
:100FAC00ED0A0319EE0ABB2F03179D0103136D08FD
:100FBC0003179E00D122073083120313FC007D30EF
:0C0FCC00FD00FD0BE72FFC0BE72F0800D9
:100FD8000D3083120317A2005D210A300317A20007
:040FE8005D2108007F
:100FEC008130831203139F008E3083169F000800FC
:1010000083120313651703179D0101309E008A1197
:10101000D1228A15831203136C080317970024301A
:1010200098000F3099008A11AA238A1503136C08BF
:1010300003179D008A1187228A15970198010313CF
:101040006C08031799008A11D5238A1501300317FC
:101050009D0001309E008A11D1228A150130831231
:1010600003179700003098000730990000309A006D
:101070000A30F40003136F08F0008A11AC228A15BD
:101080003030700703179B008A1121248A15013024
:101090008312031797000030980008309900003041
:1010A0009A000A30F40003136F08F0008A11AC2292
:1010B0008A157808F0003030700703179B008A11FA
:1010C00021248A15013083120317970000309800FD
:1010D0000930990000309A003A309B008A1121248F
:1010E0008A150130831203179700003098000A30E8
:1010F000990000309A000A30F40003136E08F000E3
:101100008A11AC228A153030700703179B008A11B0
:1011100021248A15013083120317970000309800AC
:101120000B30990000309A000A30F40003136E0867
:10113000F0008A11AC228A157808F0003030700770
:1011400003179B008A1121248A150130831203178B
:101150009700003098000C30990000309A003A3027
:101160009B008A1121248A150130831203179700EE
:10117000003098000D30990000309A000A30F400D9
:1011800003136D08F0008A11AC228A153030700705
:1011900003179B008A1121248A150130831203173B
:1011A0009700003098000E30990000309A000A3005
:1011B000F40003136D08F0008A11AC228A15780838
:1011C000F0003030700703179B008A1121248A1524
:1011D0000130831203179700003098000F309900F8
:1011E00000309A0020309B008A1121248A15831236
:1011F000031365136F088316EA0083126F08031741
:101200009700E03098008A1105268A15E030970093
:101210008A11D8248A153A30A2008A115D218A15D4
:101220006E088316EB0083126E0803179700E030F8
:1012300098008A1105268A15E03097008A11D82473
:101240008A153A30A2008A115D218A156D0883162D
:10125000EC0083126D0803179700E03098008A11A4
:1012600005268A15E03097008A11D8248A153B306C
:0A127000A2008A115D218A15080012
:10127A00831203171008840000080313ED007F305F
:10128A006D05F2007208F000F00CF013F00CF01388
:10129A00F00CF013F00CF0130A30F4008A11E92074
:1012AA008A150F306D05F1007108F0070317100851
:1012BA008400700880001108840000080313ED0000
:1012CA00F0306D05F2007208F000F00CF013F00C2B
:1012DA00F013F00CF013F00CF0130A30F4008A113A
:1012EA00E9208A150F306D05F1007108F007031720
:1012FA001108840070088000120884000008031393
:10130A00ED0030306D05F2007208F000F00CF013B9
:10131A00F00CF013F00CF013F00CF0130A30F40098
:10132A008A11E9208A150F306D05F1007108F0075E
:10133A00031712088400700880001308840007301D
:10134A000005F00013088400700880001408840067
:10135A0000080313ED00F0306D05F2007208F0008A
:10136A00F00CF013F00CF013F00CF013F00CF01377
:10137A000A30F4008A11E9208A150F306D05F10050
:10138A007108F00703171408840070088000150814
:10139A00840000080313ED0010306D05F200720896
:1013AA00F000F00CF013F00CF013F00CF013F00C4A
:1013BA00F0130A30F4008A11E9208A150F306D05FE
:1013CA00F1007108F00703171508840070088000FF
:1013DA001608840000080313ED00F0306D05F200D2
:1013EA007208F000F00CF013F00CF013F00CF0138C
:1013FA00F00CF0130A30F4008A11E9208A150F3034
:10140A006D05F1007108F0070317160884007008CB
:04141A008000080046
:10141E008A11BD228A15D030831203179D008A11BE
:10142E0014228A1570080313BD0003179D018A113B
:10143E0014228A1570080313BD008A11B1218A1572
:10144E008A11BD228A151130FC003A30FD00FD0BC9
:10145E002E2AFC0B2E2A0000D130831203179D007A
:10146E008A1114228A1570080313BD000430FC0083
:10147E003D30FD00FD0B412AFC0B412A000000000F
:10148E00013003179700003098008A11F1228A1557
:10149E00100884007008800001309700003098001A
:1014AE008A11F1228A15110884007008800001301B
:1014BE009700003098008A11F1228A1512088400D4
:1014CE007008800001309700003098008A11F122D8
:1014DE008A151308840070088000013097000030D0
:1014EE0098008A11F1228A15140884007008800071
:1014FE0001309700003098008A11F1228A151508E4
:10150E00840070088000970198018A11F1228A15D3
:10151E0016088400700880008A11B1218A1508000F
:10152E008312031365176C08031797000630F0003B
:10153E000030F1001008F400F5018A11AD248A156F
:10154E007008453E031798000E300318013E7107D0
:10155E0099008A11AA238A1503136C0803179D009C
:10156E008A1187228A159701980103136C080317B5
:10157E0099008A11D5238A15651703179D0102302C
:10158E009E008A11D1228A1502308312031797000A
:10159E00003098000530990000309A0020309B00F2
:1015AE008A1121248A150230831203179700003006
:1015BE0098000630990000309A000A30F4001108A5
:1015CE00F0008A11AC228A153030700703179B0089
:1015DE008A1121248A1502308312031797000030D6
:1015EE0098000730990000309A000A30F400110874
:1015FE00F0008A11AC228A157808F000303070079E
:10160E0003179B008A1121248A15023083120317B7
:10161E009700003098000830990000309A002F3063
:10162E009B008A1121248A1502308312031797001A
:10163E00003098000930990000309A000A30F4000A
:10164E001208F0008A11AC228A1530307007031789
:10165E009B008A1121248A150230831203179700EA
:10166E00003098000A30990000309A000A30F400D9
:10167E001208F0008A11AC228A157808F00030307A
:10168E00700703179B008A1121248A1502308312DA
:10169E0003179700003098000B30990000309A0025
:1016AE002F309B008A1121248A15023083120317D2
:1016BE009700003098000C30990000309A003230BC
:1016CE009B008A1121248A1502308312031797007A
:1016DE00003098000D30990000309A0030309B0099
:1016EE008A1121248A1502308312031797000030C5
:1016FE0098000E30990000309A000A30F40013085A
:10170E00F0008A11AC228A153030700703179B0047
:10171E008A1121248A150230831203179700003094
:10172E0098000F30990000309A000A30F400130828
:10173E00F0008A11AC228A157808F000303070075C
:10174E0003179B008A1121248A1583120313651334
:10175E000317110883160313E600831203171108EB
:10176E009700253098008A1105268A152530970096
:10177E008A11D8248A152F30A2008A115D218A156C
:10178E000317120883160313E700831203171208B8
:10179E009700253098008A1105268A152530970066
:1017AE008A11D8248A152F30A2008A115D218A153C
:1017BE000317130883160313E80083120317130885
:1017CE009700253098008A1105268A152530970036
:1017DE008A11D8248A15100883160313E9003B30AA
:0E17EE0083120317A2008A115D218A150800DC
:1017FC00831203136E08F000F00CF013F00CF013CE
:10180C00F00CF013F00CF0130030F100F830F0078E
:10181C000E300318013EF1077008E8007108E9006A
:10182C008A11E2208A150A12F0006F0884007008F1
:10183C0080006F0AF2000F306E05F0000030F100EE
:10184C00F830F0070E300318013EF1077008E8007D
:10185C007108E9008A11E2208A150A12F000720858
:10186C0084007008800002306F07F2006D08F000F1
:10187C00F00CF013F00CF013F00CF013F00CF01360
:10188C000030F100F830F0070E300318013EF1077C
:10189C007008E8007108E9008A11E2208A150A1222
:1018AC00F000720884007008800003306F07F200AB
:1018BC000F306D05F0000030F100F830F0070E30FD
:1018CC000318013EF1077008E8007108E9008A115D
:1018DC00E2208A150A12F000720884007008800059
:0A18EC0004306F078400800108003B
:1018F600831603130617861783126A10061B872C96
:0A1906006A1C862C872C812C080037
:10191000831203130715071407110330FB008A30E5
:10192000FC005530FD00FD0B932CFC0B932CFB0BA6
:10193000932C00000000071521300317A2008A1124
:1019400026218A1590300317A2008A1126218A15B4
:1019500005300317A2008A1126218A1513300317B8
:10196000A2008A1126218A1520300317A2008A11AD
:1019700026218A152130FC007630FD00FD0BBE2C9F
:10198000FC0BBE2C00000C300317A2008A1126218C
:101990008A158A11EE238A150230FB004530FC00BF
:1019A000A930FD00FD0BD22CFC0BD22CFB0BD22C52
:1019B000000000009D019E018A11D1228A150800B5
:1019C000831203137408003A031DEF2C7508003AC4
:1019D000031DEF2CFF30F0007F30F1004A2D831201
:1019E0000313FD01F901F8017108700403190034B3
:1019F00071087506FA00FA1BFD09FB01F51F052D9C
:101A0000F409F509F40A0319F50AF11F0C2DF00980
:101A1000F109F00A0319F10A71087504FA00FA1BBA
:101A2000212D8A1156268A157B18362DFD1F00346C
:101A3000F009F109F00A0319F10AF809F909F80A9D
:101A40000319F90A0034F51F322DF11B2E2D7108F0
:101A5000F9007008F800F101F001162DF101F00114
:101A6000F00A0034F109F009FB0A132DF80A0319F2
:101A7000F90A74087802031D162D75087902031DF2
:101A8000162DF901F801F00A0319F10AF11F162DBC
:061A90000000FF34080015
:101A960083120313D8015930A4001330BE0004305A
:101AA600C0000630BF000430C1001430CD008A11DA
:061AB60049238A15080017
:101ABC00831203136D08F000F00CF013F00CF0130C
:101ACC00F00CF013F00CF0130030F100F830F007CC
:101ADC000E300318013EF1077008E8007108E900A8
:101AEC008A11E2208A150A12F0006E088400700830
:101AFC0080006E0AF2000F306D05F0000030F1002E
:101B0C00F830F0070E300318013EF1077008E800BA
:101B1C007108E9008A11E2208A150A12F000720895
:101B2C0084007008800002306E0784008001080079
:101B3C008A11BD228A15A030831203179D008A11C9
:101B4C0014228A1570080313BD006E08F000F10111
:101B5C00700803179D008A1114228A15700803134C
:101B6C00BD00FF306D0503179D008A1114228A15E4
:101B7C0070080313BD006F0803179D008A1114220F
:101B8C008A1570080313BD008A11B1218A15113012
:101B9C00FC003A30FD00FD0BD12DFC0BD12D0000CB
:021BAC0008002F
:101BAE008A11E2208A150A128000840AE80A0319B3
:0A1BBE00E90AF003031DD72D08000B
:101BC8008A11BD228A15A030831203179D008A113D
:101BD80014228A1570080313BD006E08F000F10185
:101BE800700803179D008A1114228A1570080313C0
:101BF800BD00FF306D0503179D008A1114228A1558
:101C080070080313BD008A11B1218A158A11BD22FB
:101C18008A150430FC003D30FD00FD0B112EFC0B35
:101C2800112E00000000A130831203179D008A11B5
:101C380014228A1570080313BD0003179701980131
:101C48008A11F1228A1570080313EF008A11B12155
:0A1C58008A1583126F08F0000800DF
:101C620083160313981690308312980083168717F1
:101C7200071383128C1E402E1A08F0003A2E080019
:081C8200831203136A14080029
:10200000831203138601FD3083168600FF3083128E
:102010008500FF30831685008801FE30831287001B
:10202000C030831687008901FF308312890089142C
:102030000A12F6270A16831265130D30FB00AF3023
:10204000FC00B630FD00FD0B2328FC0B2328FB0B06
:1020500023280000891020308316990018158A154E
:102060000A1231268A110A160230FB004530FC00A4
:10207000A930FD00FD0B3A28FC0B3A28FB0B3A284F
:10208000000000000C300317A2000A125D210A169E
:102090000D30FB00AF30FC00B630FD00FD0B4E28CC
:1020A000FC0B4E28FB0B4E2800008914A030EC00DE
:1020B0002530D3008A150A1288248A110A1607309F
:1020C00083120313FB005830FC005930FD00FD0B58
:1020D0006728FC0B6728FB0B6728000000006517CA
:1020E0004030FB006A30FC009730FD00FD0B762885
:1020F000FC0B7628FB0B7628000000008A150A12DC
:102100007B248A110A16861C8A288A150A124B25F6
:102110008A110A1683126513583003179000243071
:1021200091003E30920041309300403094003F30A7
:1021300095004D3096008A150A120F228A110A1650
:102140005830831203179000243091003E309200E3
:1021500041309300403094003F3095004D30960060
:102160008A150A123D218A110A1603135808ED0038
:102170002408EE003E08EF008A150A1200208A119A
:102180000A16410803179000031340080317910033
:1021900003133F080317920003134D08031793001E
:1021A0008A150A1297228A110A162730FB000D3071
:1021B000FC002630FD00FD0BDB28FC0BDB28FB0BB5
:1021C000DB280000651265170430ED000030EE00DA
:1021D0000A128E270A1603179D0104309E000A1268
:1021E000D1220A16831203136C08031797003230AA
:1021F00098000F3099000A12AA230A1603136C08DC
:1022000003179D000A1287220A1606300313ED00F9
:102210000030EE000A128E270A1603179D010630C1
:102220009E000A12D1220A16831203136C080317A8
:1022300097002B3098000F3099000A12AA230A1633
:1022400003136C0803179D000A1287220A160A124C
:10225000EC270A168B0183168C1683121A08CE00FF
:102260000B178B17CF01D001E510D101D201DB0193
:10227000DC01DD01DE018316C001A0308312EC0019
:10228000583003179000243091003E3092004130C6
:102290009300403094003F3095004D3096008A15F1
:1022A0000A120F228A110A1658308312031790005F
:1022B000243091003E309200413093004030940031
:1022C0003F3095004D3096008A150A123D218A1143
:1022D0000A16031365175808ED002408EE003E089F
:1022E000EF008A150A1200208A110A1665131C30A5
:1022F000ED000F30EE000A12AE260A16A030EC00F8
:10230000ED010A1282260A16831203137008D900FF
:102310007108DA007008ED007108EE006C08EF003B
:102320000A1244270A16831203136517063003178F
:102330009D0004309E000A12D1220A168312031354
:102340006C0803179D000A1287220A16970198014C
:1023500003136C08031799000A12D5230A16651394
:102360003B300317A2000A125D210A1665175908AF
:102370000317900003135A080317910005309200C9
:10238000003093000A12CA260A1602308312031381
:102390008906A030EC001430ED000F30EE000A1278
:1023A000AE260A16A030EC000130ED000A1282269B
:1023B0000A16831203137008D4007108D500700840
:1023C000ED007108EE006C08EF000A1244270A16AF
:1023D000831203136517063003179D0006309E0015
:1023E0000A12D1220A16831203136C0803179D00E8
:1023F0000A1287220A169701980103136C08031723
:1024000099000A12D5230A165408031790000313E3
:1024100055080317910007309200003093000A120C
:10242000CA260A1683120313E518192A0A12EC2782
:102430000A160630FB001330FC00AD30FD00FD0B2A
:102440001F2AFC0B1F2AFB0B1F2A00000000CF0ACB
:102450000319D00A8030033AF00080305006700231
:10246000031D342A4F08FF3C0318382ACF01D0013E
:102470004F0803179000031350080317910008300A
:102480009200003093000A12CA260A168312031320
:102490006513E51E582EC030031797000A12D82482
:1024A0000A160A12EC270A1683164008523A031D30
:1024B000732A4108413A031D732A42085A3A031D00
:1024C000732A003083125E06031D682A03305D06FE
:1024D000031D732A7530ED000E30EE000A12AE2691
:1024E0000A16D101D20183164008573A031D6F2BFB
:1024F0004108503A031D6F2B4208453A031D6F2BCC
:10250000003083125E06031D872A03305D06031D1B
:102510006F2BE5100630D6000030D700803057060C
:10252000F00080307002031D972A0A30560203180B
:10253000622B65172530D30003179D0103309E00E1
:102540000A12D1220A1683120313530803179700A5
:10255000A13098000E3099000A12AA230A160630FC
:10256000F20003135608F0005708F100720803192F
:10257000BE2AF00DF10D7010FF3EB72A7008C7009B
:102580007108C8007008ED007108EE0009305307AB
:10259000EF008A150A12FE238A110A16B5012530AA
:1025A00003179D000A1287220A1601309700003097
:1025B0009800253099000A12D5230A168030570654
:1025C000F0008030023A7002031DE82A0030560203
:1025D00003185D2B0A12BD220A16A03083120317BE
:1025E0009D000A1214220A1670080313BD0006305B
:1025F000F0005608F3005708F40070080319052B83
:10260000F30DF40D7310FF3EFE2A7308C700740823
:10261000C8007408F000F101700803179D000A1249
:1026200014220A1670080313BD00FF304705031774
:102630009D000A1214220A1670080313BD00C90176
:10264000CA0180304A06F00080307002031D2A2B38
:10265000403049020318512B0630F2005608F000B2
:102660005708F100720803193A2BF00DF10D7010A4
:10267000FF3E332B4908F0074A080318013EF107D3
:102680007008CB007108CC00700803179D000A1277
:1026900014220A1670080313BD00C90A0319CA0AD6
:1026A000212B0A12B1210A162130FC007630FD00E0
:1026B000FD0B582BFC0B582B00008312D60A031974
:1026C000D70A8E2A0D30FB00AF30FC00B630FD007B
:1026D000FD0B682BFC0B682BFB0B682B0000831693
:1026E0004008523A031DC82C4108503A031DC82C1B
:1026F0004208453A031DC82C003083125E06031DB4
:10270000832B03305D06031DC82CE510D601D701CD
:1027100080305706F00080307002031D912B0A3084
:1027200056020318B82C0A12EC270A166517253032
:10273000D30003179D0103309E000A12D1220A160E
:1027400083120313530803179700B33098000E3019
:1027500099000A12AA230A160630F200031356083B
:10276000F0005708F10072080319BB2BF00DF10DB2
:102770007010FF3EB42B7008C7007108C8007008C5
:10278000ED007108EE0009305307EF000A124427EC
:102790000A1683120313B501253003179D000A1290
:1027A00087220A16013097000030980025309900E2
:1027B0000A12D5230A1680305706F0008030023AFC
:1027C0007002031DE52B003056020318B42C0A12C8
:1027D000BD220A16A030831203179D000A1214228C
:1027E0000A1670080313BD000630F0005608F30007
:1027F0005708F40070080319022CF30DF40D731040
:10280000FF3EFB2B7308C7007408C8007408F00073
:10281000F101700803179D000A1214220A167008AD
:102820000313BD00FF30470503179D000A12142251
:102830000A1670080313BD000A12B1210A160A1203
:10284000BD220A16A130831203179D000A1214221A
:102850000A1670080313BD00C901CA0180304A0678
:10286000F00080307002031D372C3F3049020318FE
:102870008D2C01300317970098010A12F1220A16D5
:1028800070080313C2001030F4000030F50049084E
:10289000F0004A08F1008A150A12E0248A110A168B
:1028A0007808F0007908F10000307106031D5A2CF9
:1028B00000307006031D752C0A12EC270A16470813
:1028C000ED004808EE006C08EF008A150A12FE239E
:1028D0008A110A166C08031797000A12D8240A16E0
:1028E0000930A2000A125D210A164208ED006C08A8
:1028F000EE008A150A125E258A110A166C08031763
:1029000097000A12D8240A162030A2000A125D216C
:102910000A16C90A0319CA0A2E2C0317970198012F
:102920000A12F1220A1670080313C2007008ED00A3
:102930006C08EE008A150A125E258A110A166C08C8
:10294000031797000A12D8240A160A12B1210A1690
:102950002130FC007630FD00FD0BAC2CFC0BAC2CC8
:1029600000000A12EC270A16D60A0319D70A882B88
:102970000A12EC270A160D30FB00AF30FC00B6300F
:10298000FD00FD0BC12CFC0BC12CFB0BC12C00006E
:1029900083164008533A031D042D4108543A031D81
:1029A000042D4208413A031D042D003083125E06B7
:1029B000031DDC2C03305D06031D042D8C30ED005F
:1029C0000E30EE000A12AE260A1665172530D30027
:1029D00003179D0103309E000A12D1220A168312AA
:1029E0000313530803179700C53098000E30990061
:1029F0000A12AA230A160313530803179D000A128A
:102A000087220A160313E51483164008483A031D6B
:102A1000432D4108413A031D432D42084C3A031D02
:102A2000432D003083125E06031D182D03305D0612
:102A3000031D432D65172530D30003179D01033077
:102A40009E000A12D1220A16831203135308031799
:102A50009700E73098000E3099000A12AA230A1650
:102A60000313530803179D000A1287220A16013028
:102A700097000030980003135308031799000A12B7
:102A8000D5230A16E51083164008523A031D502E2E
:102A90004108453A031D502E42084C3A031D502E62
:102AA000003083125E06031D572D03305D06031DA3
:102AB000502EE51065172530D30003179D01033014
:102AC0009E000A12D1220A16831203135308031719
:102AD0009700D63098000E3099000A12AA230A16E1
:102AE0000313530803179D000A1287220A160313C3
:102AF000651306305102F3000030031C013E520200
:102B0000F4007308F0007408F100F10CF00CF113FC
:102B10007008CB007108CC007008ED007108EE0061
:102B20005308EF000A1244270A16831203135308AE
:102B3000031797000A12D8240A160A12EC270A165D
:102B40002530D300C901CA0180304A06F000803028
:102B50007002031DAD2D053049020318CE2D490822
:102B6000ED004A08EE008A150A12E4258A110A16B9
:102B70007008EB007008ED005308EE008A150A1289
:102B80005E258A110A165308031797000A12D824E3
:102B90000A160313C90A0319CA0AA42D0A12EC273C
:102BA0000A162530D3000630C9000030CA004A0892
:102BB0005202031DDD2D49085102031C502E063020
:102BC0004902F3000030031C013E4A02F40073087E
:102BD000F0007408F100F10CF00CF113711BF11707
:102BE0007008CB007108CC007008013EED00003089
:102BF0000318013E7107EE005308EF000A12442744
:102C00000A16831203135308031797000A12D824D5
:102C10000A160930A2000A125D210A164908ED00C1
:102C20004A08EE008A150A12E4258A110A1670086D
:102C3000EB00C90A0319CA0A4908ED004A08EE0068
:102C40008A150A12E4258A110A167008F300F201A7
:102C50006B087207F00073080318013EF10070085A
:102C6000D4007108D5007008ED007108EE0053081B
:102C7000EF000A1244270A1683120313530803179E
:102C800097000A12D8240A160930A2000A125D2100
:102C90000A160A12EC270A16C90A0319CA0AD72DFE
:102CA0008316C0018312E512DD01DE01DB01DC01C8
:102CB000E51CD42E09300317A2000A125D210A1662
:102CC00065172530D30003179D0102309E000A12BC
:102CD000D1220A16831203135308031797000830F2
:102CE00098000F3099000A12AA230A1603135108FC
:102CF000ED005208EE000B305307EF000A12442794
:102D00000A1683120313530803179D000A12872221
:102D10000A16013097000030980003135308031778
:102D200099000A12D5230A16FF305405F0007008E6
:102D3000EB005108ED005208EE007008EF008A1514
:102D40000A129E258A110A162130FC007630FD00F9
:102D5000FD0BA82EFC0BA82E00008312D10A03192C
:102D6000D20A00305405F3005508FF39F400740806
:102D7000F000F1017008EB005108ED005208EE0080
:102D80007008EF008A150A129E258A110A16213052
:102D9000FC007630FD00FD0BCB2EFC0BCB2E000093
:0C2DA0008312D10A0319D20A4029D52E53
:101C8A00443469346D3461346E3400344C34753400
:101C9A006E346434693400344D34613472346434DB
:101CAA00693400344D346534723463347234003428
:101CBA004A346534753464346934003456346534CE
:101CCA006E34643472340034533461346D346534A0
:101CDA0064340034003400340034003400340034F6
:101CEA000D340A34523441345A3420344934643479
:101CFA007834203473346134763465344534653449
:0E1D0A00703472346F346D340D340A3400348A
:101D18000D340A3453345434413452345434203456
:101D280073346134763465344534653470347234D0
:0A1D38006F346D340D340A340034AA
:101D42004134643472342E3457342034503467347E
:101D520065343D342034203420342034203420347F
:041D620020340034F5
:101D66004134643472342E3452342034503467345F
:101D760065343D342034203420342034203420345B
:041D860020340034D1
:101D8A005334543441345234543420347334613427
:101D9A007634653445346534703472346F346D3456
:021DAA00003403
:101DAC004C34653463347434753472346534203493
:101DBC0045344534703472346F346D342E342034E1
:021DCC000034E1
:101DCE00533454344F3450342034733461347634B5
:101DDE002F34453465346534703472346F346D3459
:021DEE000034BF
:101DF00030343134323433343434353436343734A7
:101E0000383439344134423443344434453446342C
:101E10004E3465347834743420344934643478343E
:081E20003D342034203400346D
:101E2800203441344434433431343D342034003494
:101E3800203441344434433430343D342034003485
:0E1E4800543469346D3465343A342034003437
:0E1E560041344434433431343D3420340034BC
:0E1E640041344434433430343D3420340034AF
:1030000000340034003400340034003400345F34C1
:1030100000340034003407340034073400341434EE
:103020007F3414347F34143424342A347F342A34E3
:10303000123423341334083464346234363449345B
:103040005534223450340034053403340034003411
:1030500000341C34223441340034003441342234EE
:103060001C340034143408343E3408341434083426
:1030700008343E34083408340034503430340034DA
:103080000034083408340834083408340034603418
:1030900060340034003420341034083404340234F2
:1030A0003E345134493445343E34003442347F3464
:1030B000403400344234613451344934463421348C
:1030C000413445344B3431341834143412347F34A1
:1030D0001034273445344534453439343C344A348B
:1030E00049344934303401347134093405340334FB
:1030F0003634493449344934363406344934493451
:1031000029341E340034363436340034003400346C
:103110005634363400340034083414342234413404
:10312000003414341434143414341434003441345A
:10313000223414340834023401345134093406344E
:1031400032344934793441343E347E3411341134CC
:1031500011347E347F3449344934493436343E3472
:1031600041344134413422347F34413441342234B7
:103170001C347F3449344934493441347F34093470
:103180000934093401343E344134493449347A3401
:103190007F340834083408347F34003441347F34B9
:1031A000413400342034403441343F3401347F34DE
:1031B00008341434223441347F34403440344034B1
:1031C00040347F3402340C3402347F347F3404348E
:1031D000083410347F343E344134413441343E3479
:1031E0007F3409340934093406343E3441345134CF
:1031F00021345E347F34093419342934463446345A
:103200004934493449343134013401347F34013490
:1032100001343F344034403440343F341F34203490
:10322000403420341F343F344034383440343F3449
:103230006334143408341434633407340834703479
:10324000083407346134513449344534433400344C
:103250007F344134413400340234043408341034AF
:1032600020340034413441347F3400340434023497
:103270000134023404344034403440344034403467
:1032800000340134023404340034203454345434CF
:10329000543478347F344834443444343834383403
:1032A000443444344434203438344434443448348A
:1032B0007F343834543454345434183408347E341D
:1032C0000934013402340C345234523452343E3412
:1032D0007F340834043404347834003444347D3486
:1032E000403400342034403444343D3400347F349E
:1032F0001034283444340034003441347F344034B2
:1033000000347C3404341834043478347C34083485
:103310000434043478343834443444344434383451
:103320007C3414341434143408340834143414340D
:1033300018347C347C34083404340434083448347D
:10334000543454345434203404343F3444344034FA
:1033500020343C344034403420347C341C34203419
:10336000403420341C343C344034303440343C3419
:10337000443428341034283444340C345034503419
:1033800050343C344434643454344C344434003485
:103390000834363441340034003400347F3400348F
:1033A00000340034413436340834003410340834E6
:1033B0000834103408347834463441344634783490
:02400E00A62BDF
:020000040000FA
:1042000031003600460038003700370020007700C4
:10421000690074006800200042006F006F007400A5
:104220006C006F0061006400650072002000650092
:104230006E00200030007800310046003200380067
:1042400051003D00310030004D0048007A00200050
:10425000310039003200300030002000620064007C
:10426000730020000D000A000000FF00FF00FF00A7
:10427000FF00FF00FF00FF00FF00FF00FF00FF0046
:10428000FF00FF00FF00FF00FF00FF00FF00FF0036
:10429000FF00FF00FF00FF00FF00FF00FF00FF0026
:1042A000FF00FF00FF00FF00FF00FF00FF00FF0016
:1042B000FF00FF00FF00FF00FF00FF00FF00FF0006
:1042C000FF00FF00FF00FF00FF00FF00FF00FF00F6
:1042D000FF00FF00FF00FF00FF00FF00FF00FF00E6
:1042E000FF00FF00FF00FF00FF00FF00FF00FF00D6
:1042F000FF00FF00FF00FF00FF00FF00FF00FF00C6
:10430000FF00FF00FF00FF00FF00FF00FF00FF00B5
:10431000FF00FF00FF00FF00FF00FF00FF00FF00A5
:10432000FF00FF00FF00FF00FF00FF00FF00FF0095
:10433000FF00FF00FF00FF00FF00FF00FF00FF0085
:10434000FF00FF00FF00FF00FF00FF00FF00FF0075
:10435000FF00FF00FF00FF00FF00FF00FF00FF0065
:10436000FF00FF00FF00FF00FF00FF00FF00FF0055
:10437000FF00FF00FF00FF00FF00FF00FF00FF0045
:10438000FF00FF00FF00FF00FF00FF00FF00FF0035
:10439000FF00FF00FF00FF00FF00FF00FF00FF0025
:1043A000FF00FF00FF00FF00FF00FF00FF00FF0015
:1043B000FF00FF00FF00FF00FF00FF00FF00FF0005
:1043C000FF00FF00FF00FF00FF00FF00FF00FF00F5
:1043D000FF00FF00FF00FF00FF00FF00FF00FF00E5
:1043E000FF00FF00FF00FF00FF00FF00FF00FF00D5
:1043F000FF00FF00FF00FF00FF00FF00FF00FF00C5
:00000001FF
